:020000040008F2
:0400000018F09FE570
:04002000880008004C
:100040000120704770B50E4E0E4C82B03500361D43
:1000500005E00100306800F0CBF80C350C36A54205
:1000600009D2706831682A688842F2D1306800216C
:1000700000F0CCF8F1E702B070BC01BC0047C0460C
:10008000300208003C02080000000FE11F00C0E33E
:10009000120080E300F021E114D09FE51F00C0E3CF
:1000A0001F0080E300F021E108D09FE508009FE5F4
:1000B00010FF2FE14002010000020100C000080013
:1000C00001C08FE21CFF2FE1044C054D054E064F89
:1000D000AE462047002809D0BE4630474100080000
:1000E000D500080045000800ED000800044C054D4F
:1000F0000020AE462047044C044DAE462047000089
:1001000011010800F7000800E101080025020800BD
:1001100000B500F015F800F023F800F043F80749A7
:100120000870064800780028F7D00448007800F0EE
:100130002DF82A2000F02AF8EFE7C0460000010061
:100140000448012101600448022101600348F421B0
:10015000016070470404FFFF0804FFFF0C04FFFF69
:1001600007481121016007488021016015482321BB
:1001700001600548002101600248032101607047C9
:1001800004F4FFFF0C07FFFF0407FFFF00B50C4955
:1001900009684906FBD50B490006000E086001BC42
:1001A0000047000000B506480068C00704D50548B0
:1001B00000680006000E00E0002002BC08470000B6
:1001C0001407FFFF0007FFFF7047000010B582B063
:1001D0000400009469460120FFF7F6FFF9E70000EC
:1001E00000B581B000F01EF801B001BC004700006E
:1001F00010B40300002A05D00C78491C1C705B1C4D
:10020000521EF9D110BC00B0704700000906090E5B
:100210000300002A03D019705B1C521EFBD100B0F2
:1002200070470000014CA64620470000CD010800A1
:0C023000010000000000010000000100BF
:0400000500080000EF
:00000001FF
